:100000000000000000000528090007309F0083164B
:100010009F01DA3086008A018312002A820082075B
:1000200030340134003418340034003400340034E7
:1000300000349B34F634933441345D3467340734F0
:10004000E23403343D344D34B934CA34103491347D
:10005000593407344C346134733465347234313478
:1000600041340F344734723461346D346C34693444
:10007000633468342634423465346E3473346F34F8
:100080006E34BD0A90303D020319BD014C194D2854
:100090000230BF00BF0B4A2858283D08031D5428D2
:1000A00086160000000058283D0820020319861219
:1000B0000C1960280C30BF00BF0B5C2800008C2896
:1000C0000C111508BF002830260784003F08831351
:1000D00080001608BE003E08BF002F3026078400AF
:1000E0003F08831380000C187A28000000000000ED
:1000F00000008028BE1F7E28000080280C10A50A62
:100100002508BF003630260784003F08831380008F
:1001100007302602031DA60A00308A002308820742
:100120009928A228B128BE28F028FF280C291929CF
:1001300026294C11CC110D30BF00BF0B9D280000AB
:1001400000002F29061BA828000000000000AC2892
:100150000230A300061410140C30BF00BF0BAE28F1
:100160002F29061FB5280000B7280330A3000C3044
:10017000BF00BF0BB928000000002F29061BC528AF
:100180000D30BF00BF0BC228EF281010061004303E
:10019000A3000C18CD280000CF280C10A50A1508C4
:1001A000BF002830260784003F088313800016080C
:1001B000BF002F30260784003F08831380002508E6
:1001C000BF003630260784003F08831380000730C5
:1001D00026020319FF30031D260AA700A6012F29B6
:1001E000061FF628000000000000FA280530A300D2
:1001F0002208A0000C30BF00BF0BFC282F29061BD3
:100200000329000005290630A3000C30BF00BF0BF6
:100210000729000000002F29061F102900001229BD
:100220000730A3000C30BF00BF0B142900000000F2
:100230002F29061B1D2900001F290830A3000C30A0
:10024000BF00BF0B2129000000002F29061FA301BA
:100250000D30BF00BF0B2A29000000002F290C1809
:100260003329000035290C10A50A4B30BF00BF0B05
:100270003729000000000034861C402941203C2919
:100280004C10412041204120C2010830C3004120D0
:100290000310C20C8618C21741204120C30B472906
:1002A00041204208C1000034061141204120412074
:1002B0000830C500441C0611441806150310C40C70
:1002C000412041204120C50B5A29061541204120DB
:1002D00041200034A6010730260203188629C601F2
:1002E000363026078400460883138000C6012F306D
:1002F00026078400460883138000C601283026079D
:100300008400460883138000A60A6B29A6010034E6
:10040000C801C90106150E30A0000530A100113049
:10041000A2004C11CC110610A301A5016A211012F3
:1004200090129011901010108B0197013C214108FF
:10043000C70002308A00470ECB00CB0C4B0C0339AF
:100440008207252AA42AA42AA52A02308A00470C5A
:10045000CB00CB0C4B0C1F398207352A852AA32AE7
:10046000A32AA32AA32AA32AA32A02308A00073098
:1004700047058207422A422A472A562A6D2A6F2AAE
:10048000732A772A471C061047180614842A0F304F
:100490002705CA00861D4A16061BCA16861B4A1760
:1004A000CC19CA174A08C4005421842A36302607BA
:1004B000840083130008C40054212F3026078400D1
:1004C00083130008C40054212830260784008313B6
:1004D0000008C4005421A60A842A4C11842A4C1511
:1004E0002108A000842A4C152208A000842A6A2131
:1004F000CC154C152108A0000130A3000430970052
:100500000C118E018F01A501A32A02308A00073049
:1005100047058207922A962A9A2A9E2AA22AA22A66
:10052000A22AA22A3C214108A100A22A3C2141087A
:10053000A200A22A2108C4005421A22A2208C40031
:100540005421A22AA32A0F2B0F2B02308A00470C1A
:10055000CB00CB0C4B0C073982070F2B0F2B0F2B2B
:100560000F2B0F2BB52AC52AE12A07304705CB00F0
:1005700007304B02031DC42ACA014C18CA14CC18F8
:100580004A144A08C40054210F2B02308A00073055
:1005900047058207D22AD22AD22AD22AD92AD92A90
:1005A000DD2ADD2A4C10C7184C14CC104718CC1487
:1005B000E02ACC104718CC14E02A4C1047184C14F1
:1005C0000F2B02308A00073047058207EE2AEF2AF8
:1005D000F02AF32AF62A052B072B0C2B0F2B0F2BB7
:1005E000C40154210F2BC40154210F2B3030490278
:1005F0000318C901490A8A010F20C4005421C90AFD
:10060000303049020318C9010F2BC9010F2B4808CC
:10061000C4005421C8010F2B480A031DC80A162A1A
:02400E00293F48
:00000001FF
